:040000000A163F2F6E
:08000800FF00030E8316031331
:10001000ED000A0EEE00040EEF008A110A16812F81
:10002000C00B10280800BD08031D17280800F93070
:1000300000000000000000000000000000000000C0
:10004000FF3E031D18280000000000000000000013
:100050000000000000000000BD0B17280800C108C8
:10006000031D3328080005300000FF3E031D34281F
:1000700000000000C10B33280800EC08031D4328D2
:10008000ED080319080020306C026D0803185A2887
:10009000031D5A2861126C08EE0014186116031033
:1000A000970C960C950C940CEE03031D4D28611AC9
:1000B000141408001408150416041704FF39031952
:1000C0000800013094009501960197010800831201
:1000D0000317EE014030EF00A508031D7128013021
:1000E000EE00EE08031D87282508033A031D7A2831
:1000F000EF0187287F30EF00AB080319842825081B
:10010000023A0319EF01872825030319EF011808A4
:1001100083169200831219088316930083121A081B
:100120008316940083121B088316950083126F08B0
:10013000831696009701980199018312EF1FA42856
:1001400083169703980399038316160892071708D6
:100150000318170F930718080318180F94071908A6
:100160000318190F95077F30831218058316900026
:1001700000307E02031DBE28FD307D02031C5B297A
:100180007D08FD3C7E080318031DFE1BC828D028EF
:10019000FD307D0603197E08031DE828951FE82819
:1001A00028308312A604EF08031DE0287F309A0050
:1001B000FF30980099009B01FE30FD00FE01080011
:1001C000FF30FD00FE01980199019A019B01080092
:1001D000FE1F5B29970183122403031DF128831658
:1001E000970A831696017E08803A9B007F301B0297
:1001F000031DFC28FF307D02031C960A9A01960815
:1002000003199708031D9A0A803015059800990173
:10021000990A9808031D19109101990803199A0861
:10022000031D910AFD080319FE0803194C297D09D5
:1002300096007E099700960A0319970A2030160245
:1002400017080318252903192729971F3F29181074
:100250007D099900990A8312181C302983161814F5
:10026000031083129B0C9A0C990C980C831699031B
:10027000031D2B29181C4C29831218144C29831296
:10028000180819041A041B04FF3903194C290130FA
:10029000980099019A019B01FD01FE017F308312B4
:1002A000180583169000910803195B29900803191B
:1002B0005B2983122616831690080319612983127D
:1002C000A61683126F08831696009701980199016C
:1002D0008312EF1F6F2983169703980399038316E0
:1002E00016088312980783161708031C7A29170F1C
:1002F0007A297C298312990783161808031C8329FD
:10030000180F8329852983129A0783161908031C5D
:100310008C29190F8C298E2983129B07073083168D
:100320009600960803199D29031083129B0C9A0CC2
:10033000990C980C83169603912940301006031DE2
:10034000A5298312EE08031D18108312180819043A
:100350001A041B04FF39031D0800FD01FE010800FB
:10036000831203171B1CB8290230FD070318FE0A6D
:100370009A1FBE29FD0A031DBE29FE0A7D089B00A7
:1003800003109B0C9A137D189A17AB08031D9B173B
:100390000800403083120317E60083169001910194
:1003A000920193018312980199019A019B016608B9
:1003B000E700E603E7080319372A0310980D990DA3
:1003C0009A0D9B0D8316931FE729831218140310AF
:1003D0008316900D910D920D930D8312971F2E2A67
:1003E00010088316900783121108031CFA29110FB5
:1003F000FA29FC298316910783121208031C032A89
:10040000120F032A052A8316920783121308031C6E
:100410000C2A130F0C2A0E2A831693078312130833
:1004200083161302031D242A831212088316120254
:10043000031D242A8312110883161102031D242A86
:10044000831210088316100203182E2A8312980AAA
:100450000319990A03199A0A03199B0A83129B1B11
:10046000372A0310940D950D960D970DD729FE018F
:1004700020306602FD00031CFE03E61BFE0383160C
:100480001008110412041304FF3903190800831221
:100490001814080083120317100898001108990017
:1004A00012089A0013089B002A0829060319732AC8
:1004B0001408003CEC000030ED00EE00EF001508E1
:1004C000031C150FED021608031C160FEE02170889
:1004D000031C170FEF026C0894006D0895006E085E
:1004E00096006F0897001408980715080318150F51
:1004F000990716080318160F9A0717080318170FFD
:100500009B07AC01180819041A041B04FF39031DCA
:1005100008000130AC000800E801EB01EC016208C2
:10052000E9006308EA00681A0800641C9D2A69084B
:10053000EB076A0803186A0FEC070310E50CE40CDC
:100540000310E90DEA0DE80A932AE601E701E90143
:10055000EA01E801681A08000310E90DEA0DE20D4E
:10056000E30DE60DE70D65086702031DB92A64086F
:100570006602031CC22A6408E6026508031CE7033E
:10058000E7026914E80AAA2A831203171808190453
:100590001A041B04FF390319D92A1B1B0800031076
:1005A000980D990D9A0D9B0DFD080319FE03FD038F
:1005B000CD2AFD01FE0108008316031309108312E2
:1005C000091001300317C00010203E1CEA2A8316D0
:1005D000031309143C3083120317C0001020831644
:1005E000031309140A3083120317C00010200800F7
:1005F0008316031309108312091001300317C0007A
:1006000010208316031309140A3083120317C00045
:1006100010200130031309050317BF003230C0005A
:1006200010203F08C0000800831603130510831232
:10063000051001300317C00010203E1C222B83162A
:10064000031305143C3083120317C00010208316D7
:10065000031305140A3083120317C000102008008A
:100660008316031305108312051001300317C00011
:1006700010208316031305140A3083120317C000D9
:1006800010200130031305050317BF003230C000EE
:1006900010203F08C0000800580890005908910039
:1006A0005A089200921393015B08A700A713031046
:1006B000A70DDA1B2714A901DB1F602B0130A9004D
:1006C000DD0196302702DC00031CDD0380302702A9
:1006D000DE005E08153C0318D92BDE1BD92B5E0803
:1006E0001D3C0318A32BDE1BA32B5808003C031D45
:1006F000852B5908003C031D852B5A08003C031D1F
:10070000852B5B08CF3C03199D2B2614A9080319E0
:10071000962B5E087F3ADE1B9D2B031D9D2B100838
:10072000110412041304FF3903199D2B7F30E600D6
:10073000FF30E300E400E5000800E301E401E50127
:100740008030E60008001630DE0292175E08E700EF
:10075000E7080319B22B0310900D910D920D930D24
:10076000E703A82BA9080319D02B1008003CE700C9
:100770000030E800E900EA001108031C110FE8024C
:100780001208031C120FE9021308031C130FEA02DC
:100790006708900068089100690892006A08930051
:1007A0001008E3001108E4001208E5001308E60051
:1007B00008007E3027020318F72BA7080319E12B46
:1007C000E82B1008110412041304FF390319EE2B4F
:1007D0000130E700E801E901EA01F22BE701E80155
:1007E000E901EA01DF01E001E101E201262C9217B3
:1007F0001008E7001108E8001208E9001308EA00F1
:100800001F305C05EB00EB0803190D2C0310E70DFE
:10081000E80DE90DEA0DEB03032C1008DF001108C9
:10082000E0001208E1001308E200DC09DD09DC0A3F
:100830000319DD0A5C08EB00EB080319262C620D96
:10084000E20CE10CE00CDF0CEB031C2C67086804E5
:1008500069046A04FF39031DA616A508031D6E2C42
:10086000EA1F4F2CDF0A0319E00A0319E10A0319F2
:10087000E20A6708EB006808EC006908ED006A0806
:10088000EE000310EB0DEC0DED0DEE0D6B086C049E
:100890006D046E04FF39031D4F2CFE30DF05A908DF
:1008A0000319B02C5F08003CEB000030EC00ED00B9
:1008B000EE006008031C600FEC026108031C610F6E
:1008C000ED026208031C620FEE026B08DF006C0889
:1008D000E0006D08E1006E08E200B02CEB01670853
:1008E000680469046A04FF39031D6B14A90803191D
:1008F000A22C2503031D862CEB080319862CDF0A86
:100900000319E00A0319E10A0319E20A5F08003C2F
:10091000EC000030ED00EE00EF006008031C600FFB
:10092000ED026108031C610FEE026208031C620FF6
:10093000EF026C08DF006D08E0006E08E1006F0850
:10094000E200B02C2508023A031DB02CEB08031975
:10095000B02CDF0A0319E00A0319E10A0319E20ABD
:100960005F08E3006008E4006108E5006208E60053
:10097000080058089000590891005A0892009213F4
:1009800093015B08A700A7130310A70DDA1B271418
:100990005C0894005D0895005E0896009613970128
:1009A0005F08A800A8130310A80DDE1B2814A901D6
:1009B000DB1FDC2C0130A900AA01DF1FE12C013074
:1009C000AA002A082906AB006010270A0319601440
:1009D000E010280A0319E014601110081104120431
:1009E0001304FF3903196015E011140815041604E7
:1009F0001704FF390319E0156018002DE01C472D7E
:100A0000601C082D6019082D5A1B082D2614382D3E
:100A1000E01C102DE019102D5E1B102D2614382D12
:100A2000601C142D601D382DE01C182DE01D382D84
:100A3000E01D1F2DA808031D1F2D2614382D601D35
:100A4000262DA708031D262D2614382DE601E701C3
:100A50007F30E9008030E800AB08031DE917690822
:100A6000ED006808EC006708EB006608EA00080083
:100A7000E601E701C030E800FF30E9006908ED0059
:100A80006808EC006708EB006608EA0008007F30A1
:100A9000E100A708031D682D601D5E2DE601E7013A
:100AA000E901E801AB08031DE9176908ED006808D2
:100AB000EC006708EB006608EA000800E103921BFF
:100AC000692D0310900D910D920D930DE10A5F2D8C
:100AD0009217A808031D882DE01D7E2DE601E70171
:100AE000E901E801AB08031DE9176908ED00680892
:100AF000EC006708EB006608EA000800E103961BBB
:100B0000892D0310940D950D960D970DE10A7F2DFB
:100B100096170730E600E6080319952D0310900D8F
:100B2000910D920D930DE6038B2D0830E600E6083B
:100B30000319A12D0310940D950D960D970DE60345
:100B4000972DC921FD080319FE080319D52D7D092C
:100B50008312E6007E09E700E60A0319E70A20305F
:100B6000660267080318B62D0319B82DE71FC92DB3
:100B700060127D09E800E80A1818601603109B0C43
:100B80009A0C990C980CE803031DBC2D601A1814DC
:100B9000D52D180819041A041B04FF390319D52D83
:100BA0000130980099019A019B0183122708FD00EA
:100BB000FE012808FD070318FE0A6108FD02031C58
:100BC000FE031B1BEC2D0310980D990D9A0D9B0D28
:100BD000FD080319FE03FD036720B0211808E20099
:100BE0001908E3001A08E4001B08E5006508ED0099
:100BF0006408EC006308EB006208EA0008005B0888
:100C00008316990083125A08831698008312590894
:100C100083169700831258088316960019089A00C5
:100C200003109A0D981B1A141A088312E200E301AC
:100C3000FF30620603196308031D452E5B08831607
:100C4000990083125A088316980083125908831654
:100C50009700831258088316960098139901160876
:100C60008312E400831617088312E5008316180820
:100C70008312E600831619088312E70064086504EE
:100C800066046704FF39031D8B2E5F0883169900E5
:100C900083125E088316980083125D0883169700FE
:100CA00083125C088316960019089A0003109A0DA7
:100CB000981B1A141A088312E800E901FF3068062D
:100CC00003196908031D8F2E5F088316990083128C
:100CD0005E088316980083125D08831697008312BE
:100CE0005C08831696009813990116088312EA008F
:100CF000831617088312EB00831618088312EC0082
:100D0000831619088312ED006A086B046C046D04E5
:100D1000FF3903198F2E26148316960108005B08ED
:100D200083169A0083125A08831699008312590871
:100D300083169800831258088316970080301A058E
:100D40009B008312E00183169B080319A92E8312CE
:100D5000601483125F0883169A0083125E0883165C
:100D6000990083125D088316980083125C0883162D
:100D7000970080301A059B008312E10183169B08BF
:100D80000319C42E831261148312610860060319CB
:100D9000022F5C085804EE005D085904EF005E085D
:100DA0005A048316900083125F085B048316910037
:100DB00003108312EE0DEF0D8316900D910D92012D
:100DC000920A8312EE080319E72E8316121083127B
:100DD000EF080319ED2E8316121083169008031DD9
:100DE00012109108031D121097019208031DFA2E8C
:100DF0008312E0080319FE2E8316970A831617083C
:100E00009600080083169501950A83125C08580223
:100E100003190C2F8316950183125D0859020319DB
:100E2000132F8316950183125E085A0203191A2F95
:100E30008316950183125F085B020319212F831625
:100E400095018316930183125F085B02031D322F05
:100E50005E085A02031D322F5D085902031D322F0E
:100E60005C0858020318362F8316930A831613085A
:100E7000831260068316940097019408031995085D
:100E8000031D970A17089600080061089800620879
:100E9000990063089A0064089B001808003C031D31
:100EA000632F1908003C031D632F1A08003C031D23
:100EB000632F1B08803C031D632F0130AB009E3065
:100EC000FD00FE01882FAB019B1F832F0130AB007B
:100ED0001808003CE9000030EA00EB00EC001908BB
:100EE000031C190FEA021A08031C1A0FEB021B0855
:100EF000031C1B0FEC02690898006A0899006B0834
:100F00009A006C089B009C30FD00FE01C422672003
:100F1000B0211808E5001908E6001A08E7001B08C8
:100F2000E8006808EC006708EB006608EA0065085E
:100F3000E9000800E00803199F2F8030DF065B08F6
:100F4000A700A7130310A70DDA1B2714A901DB1FA5
:100F5000AB2F0130A90058089000590891005A0899
:100F60009200921393015F08A800A8130310A80D24
:100F7000DE1B2814AA01DF1FBF2F0130AA005C0866
:100F800094005D0895005E08960096139701063060
:100F9000E800E8080319D32F0310900D910D920D6E
:100FA000930DE803C92F0630E800E8080319DF2F86
:100FB0000310940D950D960D970DE803D52F611034
:100FC000270A03196114E110280A0319E1146111B9
:100FD0001008110412041304FF3903196115E111FB
:100FE0001408150416041704FF390319E1156118D4
:100FF000FC2F8A15E11C582861168A155E1F0128EE
:101000006112E1165A1BE112611C2428E11C2428FC
:10101000611D1528E11D15282A08290603194528F0
:101020002614A908031D44284E28611D1C28E11917
:101030001C28611A26144E2861192428E11D242831
:10104000E11E442826144428611C2A28611D2A28F0
:10105000E11C4528E11C3028E11D3028611C4F2887
:10106000611C3D2861193D28E11A2614E11C442821
:10107000E1194428611A26144428E11C4428E11986
:101080004428611A26144E285A175B08EB005A08A8
:10109000EA005908E9005808E80008005E175F08F0
:1010A000EB005E08EA005D08E9005C08E800080063
:1010B0002708E200E3012808EC00ED016C08E202D9
:1010C0006D0A03186D08E30228082702031C7C2818
:1010D00027082806031DA62817081302031D7A28CF
:1010E00016081202031D7A2815081102031D7A281A
:1010F000140810020318A62813089B0012089A006F
:1011000011089900100898002708FD00FE01290821
:10111000AB001708930016089200150891001408F8
:1011200090001B0897001A089600190895001808E7
:1011300094002808A7007D08A8002A08A9002B0809
:10114000AA00E209E309E20A0319E30AA708031D5A
:10115000CF28A808031DCF288A114A22AC088A1577
:101160000319BE282A0829060319BE282503031DD2
:10117000BC280130AB00C028AB01C0282908AB0057
:101180000630EC00EC080319CC2803109B0C9A0CD9
:10119000990C980CEC03C228FD01FE010829A8084F
:1011A000031DD828E208031DD628E303E203D9284B
:1011B0009716A708031DE128E20A031DE228E30AA7
:1011C000E22893166208EC006308ED008A113D20C6
:1011D0004A22AC088A150319F5282503031DF328B4
:1011E0000130AB00F728AB01F7282908AB0027082E
:1011F000FD00FE011B1B05290310980D990D9A0D8A
:101200009B0DFD080319FE03FD038A11C42267200C
:101210008A11B0211808E4001908E5001A08E60050
:101220001B08E7006708EB006608EA006508E900AC
:101230006408E8000800CF01D001D101D201D30138
:10124000CF1A0800471C32294308D0074408031866
:10125000440FD10745080318450FD2074608031865
:10126000460FD3070310CA0CC90CC80CC70C0310D7
:10127000C30DC40DC50DC60DCF0A2029BC013B0806
:101280003C020318080064000130BD008A111320DD
:10129000BC0A8A153F2983120317980199019A0104
:1012A0009B01C701C801C901CA01CF0141129B1BA3
:1012B0009329CA1B41160310C70DC80DC90DCA0DCD
:1012C000931B47140310900D910D920D930D031075
:1012D000980D990D9A0D9B0D17084A02031D7A2946
:1012E00016084902031D7A2915084802031D7A29A8
:1012F0001408470203187E29411E8E294112140842
:10130000C7021508031C150FC8021608031C160F88
:10131000C9021708031C170FCA021814CF0A4F0876
:10132000603A031D57294708480449044A04FF3915
:10133000031D18144F08D000080083168C189D292F
:1013400083123D088D003F088C0083168C130C150A
:1013500080300B058312C0008B13553083168D002F
:10136000AA308D008C148C18B3298312C00803197D
:10137000BA298B1783160C110800BD013B088D009C
:1013800083168C130C1483120C08BD003D08BE009C
:101390000800DC08031DCE29E10108001030DE0042
:1013A0002730DF00E001D91FE52983135B1883177D
:1013B0005A088400E201620884072D308000E00AA8
:1013C000D809D909D80A0319D90ADD01D808031D9B
:1013D000F029D908031DF0290130DD00DE00DF010E
:1013E0005C0860020318402A5E08003C03185F088E
:1013F0000319402A5F085902031D002A5E0858029B
:101400000318052ADD080319312A5808E200590893
:10141000E3005E08E4005F08E5008A11A522690880
:10142000DD005D08303EE20083135B1883175A0825
:101430006007840062088000E00A5D08E200E301C2
:101440005E08E4005F08E5008C226B08E6006C088B
:10145000E7006608D8026708031CD903D9020130E7
:10146000DD005E08E2005F08E3000A30E400E50109
:101470008A11A5226908DE006A08DF008A15F029B2
:101480005C08600203184C2A83135B1883175A0800
:1014900060078400003080006008E10008008312CB
:1014A0000317BC01BD01BE0108303C020318692AC4
:1014B0008A11F8224008BE00BD080310BD0C3E088A
:1014C000003C8A150318672A80303D04BD00BC0A21
:1014D000542A3D08BF000800BD0108303D02031832
:1014E00008003C08BE008A11DC22BC080310BC0CBA
:1014F000BD0A8A156D2A8316031309140910831275
:101500000910C8300317C0008A111020C830C0006D
:101510001020C830C00010208316031309143C307B
:1015200083120317C00010200130031309050317AD
:10153000BB003B038A15031DA02A0130BC00080034
:101540008C30C0008A111020C830C0001020C83074
:10155000C0001020BC01080083120317BC01BD01AC
:10156000BE0108303C020318C62A8A113023400805
:10157000BE00BD080310BD0C3E08003C8A150318D0
:10158000C42A80303D04BD00BC0AB12A3D08BF001A
:101590000800BD0108303D02031808003C08BE00E9
:1015A0008A111423BC080310BC0CBD0A8A15CA2A70
:1015B000831603130514051083120510C830031792
:1015C000C0008A111020C830C0001020C830C000F0
:1015D00010208316031305143C3083120317C00038
:1015E00010200130031305050317BB003B038A15C8
:1015F000031DFD2A0130BC0008008C30C0008A1198
:101600001020C830C0001020C830C0001020BC011D
:1016100008000313061086100611861106128612A2
:1016200003173E0E0F39C0000F30C005401C1A2BA7
:10163000031306140317C01C1F2B03138614031770
:10164000401D242B031306150317C01D292B03135C
:1016500086150317BF0803192F2B031306160A302C
:101660000317C1008A112F20031386160A300317AF
:10167000C1002F20031386120F3003173E05C00050
:101680000A30C1002F2003130610861006118611A0
:101690000612861203178A15401C502B03130614DA
:1016A0000317C01C552B031386140317401D5A2B18
:1016B000031306150317C01D5F2B031386150317AD
:1016C000BF080319652B031306160A300317C10060
:1016D0008A112F20031386160A300317C1002F200A
:1016E000031386120A300317C1002F2008003C089C
:1016F000DA003B08D9003A08D8003908D7005A0860
:10170000DB000310DB0DD91B5B145B08C300C401B5
:10171000FF30430603194408031DA72B3C08DA00D9
:101720003B08D9003A08D8003908D700D913DA01A4
:101730005708C5005808C6005908C7005A08C8000D
:101740004508460447044804FF39031DD72B4008C9
:10175000DA003F08D9003E08D8003D08D7005A08F3
:10176000DB000310DB0DD91B5B145B08C900CA0149
:10177000FF30490603194A08031DDA2B4008DA0036
:101780003F08D9003E08D8003D08D700D913DA0138
:101790005708CB005808CC005908CD005A08CE0095
:1017A0004B084C044D044E04FF390319DA2B261460
:1017B000D70108003C08DB003B08DA003A08D900F2
:1017C0003908D80080305B05DC00C101DC08031D4E
:1017D00041144008DB003F08DA003E08D9003D080C
:1017E000D80080305B05DC00C201DC08031D421418
:1017F0004208410603191E2C3D083904CF003E085B
:101800003A04D0003F083B04D10040083C04D20019
:101810000310CF0DD00DD10DD20DD3014F085004C0
:1018200051045204FF39031D5314D801D308031D7A
:10183000C108031DD80A5808D7000800D6013D0882
:101840003902031D2E2C3E083A02031D2E2C3F08A0
:101850003B02031D2E2C40083C02031DD60AD40176
:1018600040083C02031D3E2C3F083B02031D3E2C5A
:101870003E083A02031D3E2C3D083902031CD40ADF
:1018800054084106D500D801D508031DD608031D0C
:10189000D80A5808D70008003C08A700A71303106F
:1018A000A70DBB1B2714A901BC1F582C0130A90090
:1018B000390890003A0891003B0892009213930176
:1018C0004008A800A8130310A80DBF1B2814AA01E4
:1018D000C01F6C2C0130AA003D0894003E08950002
:1018E0003F089600961397012A082906AB0041107D
:1018F000270A03194114C110280A0319C114411100
:101900001008110412041304FF3903194115C11101
:101910001408150416041704FF390319C1154118DA
:10192000932CC11CF62C411C9B2C41199B2C3B1B5E
:101930009B2C2614E72CC11CA32CC119A32C3F1BE4
:10194000A32C2614E72C411CA72C411DE72CC11CFD
:10195000AB2CC11DE72CC11DB12CA808031DB12C57
:10196000C52C411DB72CA708031DB72CD72C411D32
:10197000C12C411CC12CC11DC12CC11CC12C261461
:10198000E72C411CD72C411DD72CC701C8017F3043
:10199000CA008030C900AB08031DCA174A08CE0030
:1019A0004908CD004808CC004708CB000800C70113
:1019B000C801CA01C901AB08031DCA174A08CE00F5
:1019C0004908CD004808CC004708CB000800C701F3
:1019D000C801C030C900FF30CA004A08CE0049081B
:1019E000CD004808CC004708CB000800A808031D1C
:1019F000042DC11D042DA708031D022D411D022D1C
:101A00002614E72C2615C52CA708031D0A2D411DF9
:101A10000A2DD72C7D30C200A708031D1D2DC20A38
:101A2000C701921B1A2D0310900D910D920D930D6D
:101A3000C70A112D4708C2021E2D9217A808031DC0
:101A40002B2DC203961B2C2D0310940D950D960D76
:101A5000970DC20A222D96172708FD00FE012808BF
:101A6000FD02031CFE034208FD070318FE0A1708C7
:101A70001302031D452D16081202031D452D1508DE
:101A80001102031D452D14081002031C4A2DFD0AE6
:101A90000319FE0A4B211818981403109B0C9A0C7A
:101AA000990C980C8A116720B0211808C3001908F6
:101AB000C4001A08C5001B08C6004608CE00450829
:101AC000CD004408CC004308CB000800BC01BD0198
:101AD000BE01BF01C001C10183133A188317390841
:101AE0008400C2014208840700082D3A031D7B2DA3
:101AF0000130BC00BD003B083D020318D62D831306
:101B00003A18831739083D07840030300002031C5F
:101B1000D62D83133A18831739083D07840000082F
:101B2000393C031CD62D3E08C3003F08C4004008C2
:101B3000C5004108C6000A30C700C801C901CA0172
:101B40001B215008CB005108CC005208CD0053088F
:101B5000CE004B08BE004C08BF004D08C0004E0828
:101B6000C10083133A18831739083D0784003030C9
:101B70000002C300C401C501C6013E08C3073F08F7
:101B800003183F0FC40740080318400FC50741085A
:101B90000318410FC6074308BE004408BF004508AC
:101BA000C0004608C1003D0ABD007B2DBC080319DA
:101BB000F42D3E08003CC3000030C400C500C60040
:101BC0003F08031C3F0FC4024008031C400FC5021E
:101BD0004108031C410FC6024308BE004408BF0071
:101BE0004508C0004608C1003E08C3003F08C400C5
:101BF0004008C5004108C6000800BF08031D022EAA
:101C0000C1010800C0013B0840020318122E8313D3
:101C10003A18831739084007840080080319122EE8
:101C2000C00A032E3C0840020318182E4008BC00CE
:101C30003C083F0203181E2E3F08BC00C0013C08B0
:101C400040020318392E83133A1883173908840089
:101C50000008C20083133E1883173D088400420821
:101C60008000BD0A0319BE0AB90A0319BA0AC00ADC
:101C70001F2E3F0840020318442E83133E1883177B
:101C80003D088400003080004008C1000800C50104
:101C90000330A5003908D8003A08D9003B08DA001B
:101CA0003C08DB008A114C236308C1006408C200B1
:101CB0004108E1004208E200E301E4018A15C21F85
:101CC000632EE303E4038A1145276908CA006A0802
:101CD000CB006B08CC006C08CD00D801D901DA012B
:101CE000DB013908DC003A08DD003B08DE003C0877
:101CF000DF00FF2596088A1503199D2E83123908E7
:101D0000D8003A08D9003B08DA003C08DB004A0852
:101D1000DC004B08DD004C08DE004D08DF00013020
:101D2000E0008A119A276808C6006908C7006A0897
:101D3000C8006B08C9008A15CA2E8312C108031D8A
:101D4000AE2EC208031DAE2E83133F1883173E0824
:101D5000450784002D308000450AC5004A08D80098
:101D60004B08D9004C08DA004D08DB003908DC00CC
:101D70003A08DD003B08DE003C08DF000130E000EF
:101D80008A119A276808C6006908C7006A08C8004F
:101D90006B08C9004108D8004208D9000130DB00B7
:101DA0004E30DA000530DC008A15C9216108C30015
:101DB000C401430844020318F62E400845020318E4
:101DC000F42E83174E3084004408D8005808840746
:101DD0000008D90083133F1883173E084507840085
:101DE00059088000450AC500C40AD92E400845029A
:101DF0000318042F83133F1883173E0845078400F8
:101E00002E308000450AC500C4013D084402031875
:101E1000722F400845020318722F4608D800470861
:101E2000D9004808DA004908DB00DC01DD01203078
:101E3000DE004130DF008A11B9246A08C6006B0851
:101E4000C7006C08C8006D08C9004608D8004708DC
:101E5000D9004808DA004908DB004C236308C100B8
:101E60006408C2004108E1004208E200E301E40125
:101E70008A15C21F3D2FE303E4038A114527690831
:101E8000CA006A08CB006B08CC006C08CD0046087D
:101E9000D8004708D9004808DA004908DB004A089A
:101EA000DC004B08DD004C08DE004D08DF0001308F
:101EB000E0009A276808C6006908C7006A08C800D9
:101EC0006B08C9004108303ED80083133F188317C0
:101ED0003E084507840058088000450AC500C40A2A
:101EE0008A15052F4008450203187E2F83133F18DB
:101EF00083173E0845078400003080004508D8005D
:101F00000800BD013C08003A03198C2F013A03195F
:101F1000952F033A03199E2F8316031308140130DB
:101F2000831208050317BD00A62F83160313881418
:101F30000230831208050317BD00A62F8316031372
:101F400008150430831208050317BD003D08BE00C4
:101F5000080083160313610883120317B900BA013E
:101F6000BB013908BC003B08B9003C08BA00831625
:101F70000313600883120317B904BA083908BB00B9
:101F80003A08BC00080083120317BA017B22BC0880
:101F90008A150319CE2F0130BB000800CC30BC00DD
:101FA0006C22BE30BC006C2209303A020318E82FC4
:101FB0004F223F08B900831603138313E0308400D7
:101FC000831203173A08840739088000BA0AD42F0D
:101FD000BB01080083120317B901BA017B22CC3080
:101FE000BC008A156C224430BC006C22B9088A11EE
:101FF0000A16031D0C288A150A124F223F08B90041
:102000000430BD008A111320BA0A3A0A8A15031D4A
:10201000F62F0130BB000800BB01080075088312D1
:102020000317B900BA01BB013908BC003B08B9006D
:102030003C08BA007408B904BA083908BB003A0869
:10204000BC00080083120317BA018A150A12D822AD
:10205000BC088A110A16031930280130BB00080099
:10206000CC30BC008A150A12C922BE30BC00C9227D
:1020700009303A028A110A1603184E288A150A12E4
:10208000AC223F08B9008313743084003A088407F7
:1020900039088000BA0A8A110A163828BB010800DC
:1020A00083120317B901BA018A150A12D822CC305B
:1020B000BC008A15C9224430BC00C922B9088A1163
:1020C0000A16031D74288A150A12AC223F08B900AB
:1020D0000430BD008A111320BA0A3A0A0A16031DF9
:1020E0005E280130BB000800BB0108008316031303
:1020F0008711831287110800831603138711831237
:1021000087150800831603130711831207110800AF
:10211000831603130711831207150800BC01BC01C5
:102120003B083C020318080083133A188317390848
:102130003C07840080080319080083133A188317AA
:1021400039083C0784000008BE001030BF008A1523
:102150000A120923BC0A0A1690283908BE0010305A
:10216000BF008A150A1209230800BA08031DBB28FC
:102170008030BA00BD28C030BA0039083A07BE0026
:10218000BF018A150A1209230230BB008A153E21BD
:1021900008003908BD003A08BE003B08BF008A1598
:1021A0000A129D2108003908BB003A08BC008A15B4
:1021B0000A12BD213E08BB00BC01080083120317B0
:1021C000B901BA01D3203B08B500350834028A11A1
:1021D0000A16031C0229EF30831603130805880032
:1021E000EF30831208050317B900103039040313C8
:1021F0008800DF30831608058800DF308312080569
:1022000088004E293408E100E201E301E4010A12EA
:1022100045276908B9006A08BA006B08BB006C085A
:10222000BC003508E100E201E301E401452769084B
:10223000D8006A08D9006B08DA006C08DB0033307C
:10224000DC00DD003F30DF00F330DE000130E00075
:102250009A276808BD006908BE006A08BF006B08BD
:10226000C0008A157723D7088A110A1603194E2948
:10227000EF308316031308058800EF30831208053A
:102280008800DF30831608058800DF3083120805D8
:102290000317B900203039040313880003172F08EF
:1022A0002D02031C6A29BF3083160313080588001A
:1022B000BF30831208050317B900403039040313F7
:1022C00088007F308316080588007F308312080558
:1022D000880008002D08E100E201E301E4010A1290
:1022E00045276908B9006A08BA006B08BB006C088A
:1022F000BC002F08E100E201E301E4014527690881
:10230000D8006A08D9006B08DA006C08DB003330AB
:10231000DC00DD003F30DF00F330DE000130E000A4
:102320009A276808BD006908BE006A08BF006B08EC
:10233000C0008A157723D70803190800BF30831619
:10234000031308058800BF308312080588007F301A
:102350008316080588007F30831208050317B9002B
:10236000803039040313880008007C208A150A1283
:10237000EA273B08B2008A150A12C3273B08B200BD
:10238000A9273B08E1003C08E200E301E4018A11CF
:1023900045276908A0006A08A1006B08A2006C0824
:1023A000A3000A16762003172008B9002108BA00F6
:1023B0002208BB002308BC00BD01BE018030BF0065
:1023C0004130C0008A150A124C244B08A0004C086A
:1023D000A1004D08A2004E08A3002008B900210862
:1023E000BA002208BB002308BC000630BD00003044
:1023F000BF006030BE001430C0008A154726003090
:10240000BA006030B9001430BB0066254308AD0047
:10241000D801D901C830DA004230DB002008DC00E6
:102420002108DD002208DE002308DF008A11FF25D5
:1024300096080A160319312A00308312BA00603058
:10244000B9001430BB000530BC000030BE00603065
:10245000BD001430BF008A150A12FD258A110A1624
:10246000432A00308312BA006030B9001430BB0038
:102470000430BC000030BE006030BD001430BF002E
:102480008A150A12FD25B901BA011630BB00433086
:10249000BC002008BD002108BE002208BF002308A0
:1024A000C0008A150A127723D7088A110A16031961
:1024B000902AB9010130BA00B5202030B9008A1144
:1024C0000A16AD207430B9000A16AD206530B90087
:1024D0000A16AD206D30B9000A16AD207030B90073
:1024E0000A16AD203230B9000A16AD202030B900EE
:1024F0000A16AD202030B9000A16AD202D30B900E3
:102500000A16AD202D30B9000A16AD202D30B900C5
:102510000A16AD202D30B9000A16AD200A16BD2AC4
:10252000B9010130BA00B5202030B9008A110A166D
:10253000AD207430B9000A16AD206530B9000A1616
:10254000AD206D30B9000A16AD207030B9000A1602
:10255000AD203230B9000A16AD202030B9000A167D
:10256000AD202030B9000A16AD200030BA0060302E
:10257000B9001430BB000A168E202030B900AD20FF
:102580004330B9000A16AD202030B9000A16AD203C
:102590002030B9000A16AD200800882050203B08E2
:1025A000AE0022203B08AE000E203B08E1003C08B4
:1025B000E200E301E4010A1245276908A0006A0865
:1025C000A1006B08A2006C08A3000A168220031762
:1025D0002008B9002108BA002208BB002308BC006B
:1025E000BD01BE018030BF004130C0008A150A1213
:1025F0004C244B08A0004C08A1004D08A2004E0836
:10260000A3002008B9002108BA002208BB00230853
:10261000BC000630BD000030BF006030BE0014308A
:10262000C0008A1547260030BA006030B900143067
:10263000BB0066254308B400D801D901C830DA00D0
:102640004230DB002008DC002108DD002208DE002B
:102650002308DF008A11FF2596080A160319452B67
:1026600000308312BA006030B9001430BB0005306E
:10267000BC000030BE006030BD001430BF008A15C1
:102680000A12FD258A110A16572B00308312BA0050
:102690006030B9001430BB000430BC000030BE0014
:1026A0006030BD001430BF008A150A12FD25B90143
:1026B000BA011630BB004330BC002008BD00210821
:1026C000BE002208BF002308C0008A150A12772323
:1026D000D7088A110A160319A32BB901BA01B5202C
:1026E0002030B9008A110A16AD207430B9000A16DC
:1026F000AD206530B9000A16AD206D30B9000A165C
:10270000AD207030B9000A16AD203130B9000A167C
:10271000AD202030B9000A16AD202030B9000A16CD
:10272000AD202D30B9000A16AD202D30B9000A16A3
:10273000AD202D30B9000A16AD202D30B9000A1693
:10274000AD200A16CF2BB901BA01B5202030B9004F
:102750008A110A16AD207430B9000A16AD20653012
:10276000B9000A16AD206D30B9000A16AD207030E0
:10277000B9000A16AD203130B9000A16AD2020305C
:10278000B9000A16AD202030B9000A16AD2000307D
:10279000BA006030B9001430BB000A168E20203019
:1027A000B900AD204330B9000A16AD202030B90081
:1027B0000A16AD202030B9000A16AD200800831299
:1027C0000317B901BA01D3203B08B5003508823C94
:1027D0008A110A160318F22BB901BA013230BB0074
:1027E000BC01C92001308312B900BA018A110A164E
:1027F000D3203B08AF002F08823C031808000130AB
:10280000B900BA013230BB00BC018A110A16C920D6
:102810000800FF30BB003A08BC008A150A12812765
:102820003E08BB00BB088A110A1603191A2C013096
:10283000BC000800BC010800BA1F2D2C2D30BE00C2
:102840001030BF008A150A1209233908003CBE0067
:10285000BA090318BA0A3E08B9003908BB003A0899
:10286000BC0027303A020A16031D382C10303902FA
:10287000031C6B2CBA1B6B2CBE013B08E2003C080E
:10288000E300BC1F492CE209E309E20A0319E30A49
:10289000BE0A1030E4002730E5000A12A5226908BC
:1028A000BD000A163E1C562CBD09BD0A3D08303E2F
:1028B000BE001030BF008A150A1209233D08003CF3
:1028C0000A1603186B2C1030BB022730031C28306B
:1028D000BC02BD035E2C03303A02031D712CE830AC
:1028E0003902031CA62CBA1BA62CBF013B08E20030
:1028F0003C08E300BC1F822CE209E309E20A031949
:10290000E30ABF0AE830E4000330E5000A12A5221A
:102910006908BE000A163F1C8F2CBE09BE0A3E087D
:10292000BD003D08303EBE001030BF008A150A12BF
:1029300009233D08003C0A160318A62CE830BB0208
:102940000330031C0430BC02BD03992C3A08803AC2
:10295000BE0080303E02031DAF2C64303902031CE0
:10296000E02CBF013B08E2003C08E300BC1FBE2C8A
:10297000E209E309E20A0319E30ABF0A6430E4004A
:10298000E5010A12A5226908BE000A163F1CCA2CDE
:10299000BE09BE0A3E08BD003D08303EBE001030F4
:1029A000BF008A150A1209233D08003C0A160318C5
:1029B000E02C6430BB02BC08031CBC03BD03D42C58
:1029C0003A08803ABE0080303E02031DE92C0A30EE
:1029D0003902031C1A2DBF013B08E2003C08E3004A
:1029E000BC1FF82CE209E309E20A0319E30ABF0A53
:1029F0000A30E400E5010A12A5226908BE000A16A1
:102A00003F1C042DBE09BE0A3E08BD003D08303EF5
:102A1000BE001030BF008A150A1209233D08003C91
:102A20000A1603181A2D0A30BB02BC08031CBC038B
:102A3000BD030E2D3B08303EBE001030BF008A158E
:102A40000A120923080083160313061083120610C6
:102A500083168610831286108316061183120611C0
:102A600083168611831286118316061283120612AC
:102A700083168612831286120C300317BB008A1548
:102A80000A123E213330BE00BF0109230230BB00D1
:102A90008A153E213330BE00BF0109230230BB003E
:102AA0008A153E213230BE00BF0109230230BB002F
:102AB0008A153E212C30BE00BF0109230230BB0025
:102AC0008A153E210630BE00BF0109230230BB003B
:102AD0008A153E210C30BE00BF0109230230BB0025
:102AE0008A153E210130BE00BF0109230230BB0020
:102AF0008A153E210230BE00BF0109230230BB000F
:102B00008A153E2108000730831603139F00C0304A
:102B1000810023258A110A16DF238312B6010230B1
:102B20000317BA008A110A160924B901BC08031D4B
:102B3000391430103908031D3014301CA12D360A09
:102B4000B600B608031DB82DCD220230BA000A1611
:102B50000924B901BC08031D391430103908031DBC
:102B60003014301CB52D360AB600B5210A16362FA2
:102B70003603031D722EBA0109243C08B300B901C3
:102B8000BA01D3203B08B50033038A110A16031D8E
:102B9000D12D3503B500B901BA013508BB00BC0120
:102BA000C92001308312BA008A110A1609243C0890
:102BB000B100B901BA01D3203B08B50031038A1135
:102BC0000A16031DEB2D350AB500B901BA01350807
:102BD000BB00BC01C9208312B901BA018A110A16CF
:102BE000B5202030B9008A110A16AD207230B90024
:102BF0000A16AD206530B9000A16AD206730B9005D
:102C00000A16AD205F30B9000A16AD203130B90088
:102C10000A16AD202030B9000A16AD202030B900C8
:102C20000A16AD203508B900BA010A161C24203056
:102C3000B9000A16AD204330B9000A16AD20203085
:102C4000B9000A16AD202A30B9000A16AD2020308E
:102C5000B9000A16AD202030B9000A16AD20B9011E
:102C60000130BA000A16B5202030B9008A110A16C0
:102C7000AD207230B9000A16AD206530B9000A16D1
:102C8000AD206730B9000A16AD205F30B9000A16D2
:102C9000AD203230B9000A16AD202030B9000A1636
:102CA000AD202030B9000A16AD202F08B900BA01B6
:102CB0000A161C242030B9000A16AD204330B90092
:102CC0000A16AD202030B9000A16AD202030B90018
:102CD0000A16AD202030B9000A16AD202030B90008
:102CE0000A16AD203608023A0A16031D322FBA0121
:102CF00009243C08B3000130B900BA01D3203B08D5
:102D0000AF0033038A110A16031D8F2E2F03AF0065
:102D10000130B900BA012F08BB00BC01C920013045
:102D20008312BA008A110A1609243C08B100013046
:102D3000B900BA01D3203B08AF0031038A110A164B
:102D4000031DAB2E2F0AAF000130B900BA012F08C6
:102D5000BB00BC01C9208312B901BA018A110A164D
:102D6000B5202030B9008A110A16AD207230B900A2
:102D70000A16AD206530B9000A16AD206730B900DB
:102D80000A16AD205F30B9000A16AD203130B90007
:102D90000A16AD202030B9000A16AD202030B90047
:102DA0000A16AD203508B900BA010A161C242030D5
:102DB000B9000A16AD204330B9000A16AD20203004
:102DC000B9000A16AD202030B9000A16AD20203017
:102DD000B9000A16AD202030B9000A16AD20B9019D
:102DE0000130BA000A16B5202030B9008A110A163F
:102DF000AD207230B9000A16AD206530B9000A1650
:102E0000AD206730B9000A16AD205F30B9000A1650
:102E1000AD203230B9000A16AD202030B9000A16B4
:102E2000AD202030B9000A16AD202F08B900BA0134
:102E30000A161C242030B9000A16AD204330B90010
:102E40000A16AD202030B9000A16AD202A30B9008C
:102E50000A16AD202030B9000A16AD202030B90086
:102E60000A16AD20C830BD000A1213200330360206
:102E70000318B6010A16DE208A110A168F2DD530E6
:102E800083160313E900C430EA00BB30EB00DC30EA
:102E9000EC008312031790019101920193019401B8
:102EA000950196019701980199019A019B01A7014B
:102EB000A801FD01FE01A901AA01AB01AC019C0121
:102EC0009D019E019F01A501A601A401B701031365
:102ED0008313203084003F30DF008001840A8A1190
:102EE0000A16DF0B6D2F0317B80183160313831324
:102EF000A03084003F30DF008001840ADF0B7C2F8C
:102F0000832D831603136F0E84006E0E8A006D0EE0
:082F10008300FF0E7F0E090093
:02400E00723FFF
:00000001FF
